:020000040000FA
:02000000F629DF
:080008008C00030E8D000B1C9F
:100010000B280B102C210B1D122883120B110530FD
:1000200081001A140D0E83008C0E0C0E090082073D
:100030000000C529C829CB29CB28CE28DD28DF28F8
:10004000E928EB28ED28F228F528F828FB28FE28D7
:100050000129062908290A29820730283428382846
:1000600028080F219A14080028080C219A14080067
:1000700028081621080083120508F039850086112A
:100080000617861783160508F039850006138613B0
:100090008611831208008E0032308F0004309000E9
:1000A0000000900B50288F0B4E288E0B4C28080018
:1000B000861500008611080086138F000F0E0F3979
:1000C0008E000508F0390E04850058200F080F39FE
:1000D0008E000508F0390E048500582008008613AC
:1000E0008E000508F0398E0E0E0485005820080099
:1000F00006135C2806175C28831605080F38850050
:1001000083128617000086150000050886110F3936
:100110008E0086158E0E050886110F398E04861303
:1001200083160508F039850083120E0808000613AF
:100130007C2806177C289720803908008312972096
:100140008039031D9E2808009E20110E07390838AB
:1001500078280C3991003B2010304B2006133030AA
:100160006F2005304B2030306F2005304B20303071
:100170006F2005304B20203011046F209E20083066
:100180005C209E2001305C209E2006305C200230E6
:1001900091049E2008009E20013078289E20023085
:1001A00078280239031DD728FD309105D8289104FD
:1001B0009E2011080339043878280230D128030121
:1001C000D1280139031DE728FE309105D828910474
:1001D000D8280130E1280301E128110E04389100EC
:1001E000910EA428110EFB39EF28110E0238EF28CA
:1001F000110EFD39EF28110E0138EF28110EFE39CE
:10020000EF28183090009E2010087828203002290E
:1002100010300229183002293F39403802297F392D
:10022000803802299E2097207F39080090009E2068
:1002300010087A289E209928940094138316061695
:1002400086168312061686160608950092019301FB
:100250009601970192140800831206089506151A54
:100260003529951A9429950008009500151A6B29CF
:10027000931C542993101311931108309700131EE7
:10028000512916180800931A612912169216121E87
:100290004D290612831606128312831686168312C0
:1002A0000800121B12164729131D59299314960191
:1002B0006429931D5E29931193144D29131E080080
:1002C00064291908960093128616961F86128316C3
:1002D0008612831208000310951A0314960D970BCB
:1002E0000800131C88291310140D1606FE39031D6F
:1002F0000800161C7E29121980290800921C08008B
:1003000092151315161C08001316931E921608005A
:10031000921D0800131E8E299315080016089800D8
:1003200012179218131508009500151E0800921157
:1003300013121210951A08001214131413129314A6
:10034000080018081213121E0800131A08001217CA
:1003500012128316061683122C2118081213080095
:10036000990092129316121E0800131E08006121B4
:1003700012128316061683122C2912150800121168
:10038000080092140800921008001A119A1108002F
:100390001A159A1108009A151A11080083120611ED
:1003A0001B18061586109B18861406101B190614B8
:1003B0001E301B0784000310051E0314800D000867
:1003C00003191D14FF3A03191D109D0C9D130318EA
:1003D0009D179B0A9B1D08001D089C009B0108009F
:1003E0001A1912299A191A291C0808008316513063
:1003F000810006118610061005168312061186105C
:1004000006109A01A7019C0108309B001E30840051
:100410008001840A9B0B082A42301C21BD21083030
:10042000A920ED2000300F2181018B168B158B1731
:10043000921E1D2AF021B021392A921D9A14121FF2
:10044000392AA1219A1C312A9A10A700A71E2A2A0C
:10045000A712392A133C031C392A270817209A149B
:10046000182AA8002708023C031C392A27082C2038
:0C047000182A1A1C3D2A1A10CE21182A46
:02400E000200AE
:00000001FF
